:0200000480007A
:10000000970000009380C002F39F503097100000CB
:10001000938040FF3711111113011111730010006B
:1000200023A0000073905F306F008002732F1034A4
:10003000130F4F0073101F34732F203423A0E001DF
:1000400023A2200023A400009380C000730020306E
:1000500017150000130505FB97150000938585FB18
:10006000370610F01306C6F26306B5028326C500F4
:100070002320D600832685002320D6008326450032
:100080002320D600832605002320D6001305050172
:100090006FF09FFD370510F0130505F223200500D2
:0400A000000000005C
:10100000FFFFFFFFFFFFFFFFFFFFFFFFFFFFFFFFF0
:040000058000000077
:00000001FF
